:020000040000FA
:06000000CA3001303A286D
:08000800A000030EA100831209
:100010008B1C32288B1032181428B21C3228643002
:10002000010203183128182800001628172818285C
:1000300019281A281B281C281D281E281F283210A2
:10004000B214A810031005190314AA0DA90DA80DC8
:10005000B10B322832152A08AF002908AE00280853
:10006000AD00B21081010B11210E8300A00E200EF5
:02007000090085
:0C007400203084008001840A80300402E7
:10008000031C3C281230B100E52183160C30850595
:1000900087018312850187010730990000309A009B
:1000A000103083168E008312603083168F00831207
:1000B00000308316910000008312C830831681003F
:1000C000831231309000003083168C008312103080
:1000D0008B00BD1B7128851971286400851D6D2852
:1000E000F622DD2281018E018F010B118B100B1086
:1000F0008C018B17892032199F20B40B872803109D
:1001000085190314BA0DF0303A02031945213C2336
:100110007A286400321808000B1D08000B11B21079
:1001200032141230B100051D9A28331483160113BE
:10013000831208003310831601178312080032114E
:100140000130B7008B132030370783169B001C1437
:100150001A088312A400A500C030A5061030370786
:1001600083169B001C141A088312A3000030370763
:1001700083169B001C141A088312A2008B17331CD1
:10018000C72822090339A200A309A409A509220846
:100190002D02031D3F2923082E02031D3F29240899
:1001A0002F02031D3F2901303702031DDC283E18B2
:1001B000DC283E143F14072202303702031DE528D5
:1001C000BE18E528BE143F14162203303702031D63
:1001D000EE283E19EE283E153F1422220430370245
:1001E000031DF728BE19F728BE153F142E2205302F
:1001F0003702031D00293E1A00293E163F143D22F6
:1002000006303702031D0929BE1A0929BE163F14FC
:100210004C2207303702031D12293E1B12293E17BC
:100220003F145B2208303702031D1B29BE1B1B290C
:10023000BE173F14662209303702031D24295D18BA
:1002400024295D143F1471220A303702031D2D2921
:10025000DD182D29DD143F147C220B303702031DDD
:1002600036295D1936295D153F1487220C30370277
:10027000031D3F29DD193F29DD153F149222B70ADE
:100280000D30370203180800A2280130B600B40070
:10029000B500B70085018701B213DA228920B40BBB
:1002A0005E29031085190314BA0DF0303A020319C0
:1002B0008529B50B5E299630B5009121321D4E2956
:1002C0003211331C68292D090339AD00AE09AF097D
:1002D0002F1CB2132F1C4E29B21B4E292E184E294B
:1002E000B2178B1320303707BC002F08BB00D0217A
:1002F00010303707BC002E08BB00D0210030370774
:10030000BC002D08BB00D0218B1785018701B70ADF
:10031000B6010130B5000D303702031C4E29DD2235
:1003200008000130370203199E22023037020319F8
:10033000A322033037020319A8220430370203191D
:10034000AD22053037020319B222063037020319F5
:10035000B722073037020319BC22083037020319CD
:10036000C122093037020319C6220A3037020319A5
:10037000CB220B3037020319D0220C30370203197D
:10038000D52208003F1C08003F101030BC003E087A
:10039000BB00D0213030BC005D08BB00D02108007C
:1003A0008B133B0883161C159A0083123C08831696
:1003B0009B0055309D00AA309D009C1464009C1841
:1003C000DE291C1183128B170800831600309B0056
:1003D0001C141A088312BD00831610309B001C14D5
:1003E0001A088312BE00831630309B001C141A08B2
:1003F0008312DD00FF30C800CA15CB15CC15CD1512
:10040000CE15CF15D015D115D215D3150800C13092
:10041000BE05FF30DD055F141130C405C00000309B
:10042000C200BD185E14BD18DE140800C230BE053F
:10043000FF30DD055F140230C405C0000030C2008B
:100440005E100800C430BE05FF30DD055F140630C5
:10045000C405C0000030C2005E100800C830BE05F0
:10046000FF30DD055F141830C405C0000030C20045
:10047000BD185E14BD18DE140800D030BE05FF3074
:10048000DD055F143030C405C0000030C200BD1867
:100490005E14BD18DE140800E030BE05FF30DD0537
:1004A0005F143030C405C0002030C200BD185E1497
:1004B000BD18DE1408007F30BE050030DD05DF14F6
:1004C000C030C505C1000030C3000800BF30BE0504
:1004D0000030DD05DF143030C505C1000030C30039
:1004E00008003F30BE050130DD05DF149030C50542
:1004F000C1000030C30008003F30BE050230DD05FA
:10050000DF14C030C505C1000030C30008003F3013
:10051000BE050430DD05DF14C030C505C100003064
:10052000C30008003F30BE050830DD05DF14C030D1
:10053000C505C1000030C300080008001030850662
:100540000230870608002030850600308706080044
:10055000213085060030870608000230850602300B
:100560008706080000308506063087060800003040
:100570008506063087060800003085061830870695
:100580000800003085062130870608000030850607
:1005900009308706080000308506183087060800F5
:1005A00000308506183087060800003085061830B0
:1005B000870608003E189E2208003E180722BE1833
:1005C00016223E192222BE192E223E1A3D22BE1AA2
:1005D0004C223E1B5B22BE1B66225D187122DD1879
:1005E0007C225D198722DD1992220800B601B40130
:1005F000B5013D1CFE2ABD01BD14002BBD013D14FB
:100600003D08B6006400042B052B062B072B082B96
:10061000FF30B51B8500B51F8501B40B022BB50B50
:10062000022B0310B60CB608031D022B0030BC00D1
:100630003D08BB00D021080005125C180516DC1C23
:100640008512DC1885165C1D05105C190514DC1D6F
:100650008510DC1985145C1E87105C1A8714DC1E5B
:100660000711DC1A07155C1F07105C1B0714DC1F41
:100670008712DC1B871608008F08031908008F01FA
:1006800078308E00C80F8C2DC80A42084304031925
:100690004F2B4208C600C2014308C700C301DE1940
:1006A000782B441C782B461C692BCA1C5A2BCA0178
:1006B0004A15862B4A1D5F2BCA01CA15862BCA1DF7
:1006C000642BCA014A16862B4A1E862BCA01CA14FD
:1006D000862B4A1D6E2BCA014A16862BCA1D732B08
:1006E000CA014A16862B4A1E862BCA01CA14862BBB
:1006F000CA1C7D2BCA014A15862B4A1D822BCA01B2
:10070000CA15862B4A1E862BCA014A15DE19AF2B45
:10071000C41CAF2BC61CA02BCB1C912BCB014B15A3
:10072000BD2B4B1D962BCB01CB15BD2BCB1D9B2B76
:10073000CB014B16BD2B4B1EBD2BCB01CB14BD2BC0
:100740004B1DA52BCB014B16BD2BCB1DAA2BCB01D3
:100750004B16BD2B4B1EBD2BCB01CB14BD2BCB1C85
:10076000B42BCB014B15BD2B4B1DB92BCB01CB159E
:10077000BD2B4B1EBD2BCB014B15DE19E62B441DAB
:10078000E62B461DD72BCC1CC82BCC014C15F42BCB
:100790004C1DCD2BCC01CC15F42BCC1DD22BCC0178
:1007A0004C16F42B4C1EF42BCC01CC14F42B4C1D0A
:1007B000DC2BCC014C16F42BCC1DE12BCC014C16C0
:1007C000F42B4C1EF42BCC01CC14F42BCC1CEB2BB7
:1007D000CC014C15F42B4C1DF02BCC01CC15F42B7B
:1007E0004C1EF42BCC014C15DE191E2CC41D1E2CE6
:1007F000C61D0F2CCD1C002CCD014D155E132C2CCD
:100800004D1D052CCD01CD152C2CCD1D0A2CCD0157
:100810004D162C2C4D1E2C2CCD01CD142C2C4D1DE9
:10082000142CCD014D162C2CCD1D192CCD014D169F
:100830002C2C4D1E2C2CCD01CD142C2CCD1C232C5E
:10084000CD014D152C2C4D1D282CCD01CD152C2C5A
:100850004D1E2C2CCD014D15DE19572C5E1B572C2F
:10086000441E572C461E482CCE1C392CCE014E154A
:10087000652C4E1D3E2CCE01CE15652CCE1D432C75
:10088000CE014E16652C4E1E652CCE01CE14652C65
:100890004E1D4D2CCE014E16652CCE1D522CCE0178
:1008A0004E16652C4E1E652CCE01CE14652CCE1C2A
:1008B0005C2CCE014E15652C4E1D612CCE01CE1543
:1008C000652C4E1E652CCE014E15DE198E2CC41ED5
:1008D0008E2CC61E7F2CCF1C702CCF014F159C2C4C
:1008E0004F1D752CCF01CF159C2CCF1D7A2CCF011D
:1008F0004F169C2C4F1E9C2CCF01CF149C2C4F1DAF
:10090000842CCF014F169C2CCF1D892CCF014F1664
:100910009C2C4F1E9C2CCF01CF149C2CCF1C932CB5
:10092000CF014F159C2C4F1D982CCF01CF159C2C1F
:100930004F1E9C2CCF014F15DE19C72CDE18C72C7B
:10094000451EC72C471EB82CD01CA92CD001501511
:10095000D52C501DAE2CD001D015D52CD01DB32CCC
:10096000D0015016D52C501ED52CD001D014D52C2A
:10097000501DBD2CD0015016D52CD01DC22CD0013D
:100980005016D52C501ED52CD001D014D52CD01CEF
:10099000CC2CD0015015D52C501DD12CD001D01508
:1009A000D52C501ED52CD0015015DE19002DDE1887
:1009B000002DC51E002DC71EF12CD11CE22CD1012B
:1009C00051150E2D511DE72CD101D1150E2DD11D24
:1009D000EC2CD10151160E2D511E0E2DD101D1142A
:1009E0000E2D511DF62CD10151160E2DD11DFB2CB3
:1009F000D10151160E2D511E0E2DD101D1140E2DE7
:100A0000D11C052DD10151150E2D511D0A2DD101DD
:100A1000D1150E2D511E0E2DD1015115DE193A2D75
:100A2000DE183A2D451F3A2D471F2B2DD21C1C2DA9
:100A3000D2015215DE13482D521D212DD201D2159F
:100A4000482DD21D262DD2015216482D521E482D5A
:100A5000D201D214482D521D302DD2015216482DEC
:100A6000D21D352DD2015216482D521E482DD201CD
:100A7000D214482DD21C3F2DD2015215482D521DA3
:100A8000442DD201D215482D521E482DD2015215A7
:100A9000DE19752DDE18752DDE1B752DC51F752D04
:100AA000C71F662DD31C572DD3015315832D531DFE
:100AB0005C2DD301D315832DD31D612DD301531686
:100AC000832D531E832DD301D314832D531D6B2DE2
:100AD000D3015316832DD31D702DD3015316832DAF
:100AE000531E832DD301D314832DD31C7A2DD30110
:100AF0005315832D531D7F2DD301D315832D531EE5
:100B0000832DD3015315C2214008C4004108C500FC
:100B10005E18DE145E1CDE104808C9000C304A0561
:100B2000031D05120C304B05031D85120C304C05BE
:100B3000031D05100C304D05031D85100C304E05AE
:100B4000031D87100C304F05031D07110C30500595
:100B5000031D07100C305105031D87120C30520580
:100B6000031D07120C305305031D871149080E029F
:100B70000318E62D12304A05031D051612304B05E9
:100B8000031D851612304C05031D051412304D054A
:100B9000031D851412304E05031D871412304F05B6
:100BA000031D071512305005031D0714123051059F
:100BB000031D871612305205031D07161230530508
:100BC000031D8715FF304802031908008F08031D15
:100BD0000800892049080E02031CE62D18304A053A
:100BE000031D051206304A05031D051618304B0576
:100BF000031D851206304B05031D851618304C0564
:100C0000031D051006304C05031D051418304D0555
:100C1000031D851006304D05031D851418304E0543
:100C2000031D871006304E05031D871418304F052D
:100C3000031D071106304F05031D07151830500519
:100C4000031D071006305005031D07141830510509
:100C5000031D871206305105031D871618305205F3
:100C6000031D071206305205031D071618305305E1
:0E0C7000031D871106305305031D871508006C
:020C7E00003440
:020C800000343E
:084000000200030007000100AB
:02400E00CC33B1
:10420000010003000300030003000200020002009B
:104210000200000000000000000003000300030093
:10422000410000000000000000000000000000004D
:104230000000C000C000C000C000C000C000C0003E
:10424000FF00C300F300CF00FF00C300F300CF0066
:10425000FF00C300F300CF00FF00C300F300CF0056
:104260000000FF00FF00FF00FF00FF00FF00FF0055
:10427000FF00FF00FF00FF00FF00FF00FF00FF0046
:10428000FF000300FF00FF00FF00FF00FF00FF0032
:10429000FF00FF00FF00FF00FF00FF00FF00FF0026
:1042A000FF00C000FF00FF00FF00FF00FF00FF0055
:1042B000FF00FF00FF00FF00FF00FF00FF00FF0006
:1042C000FF00FF00FF00FF00FF00FF00FF00FF00F6
:1042D000FF00FF00FF00FF00FF00FF00FF00FF00E6
:1042E000FF00FF00FF00FF00FF00FF00FF00FF00D6
:1042F000FF00FF00FF00FF00FF00FF00FF00AA001B
:00000001FF
